S3150800000030280020690200085B170008531700080B
S315080000105717000809070008E54300080000000014
S31508000020000000000000000000000000813F0008FA
S315080000301507000800000000750600089102000870
S31508000040930200089302000893020008930200082E
S31508000050930200089302000893020008930200081E
S31508000060930200089302000893020008930200080E
S3150800007093020008930200089302000893020008FE
S3150800008093020008930200089302000893020008EE
S3150800009093020008930200089302000893020008DE
S315080000A093020008930200089302000893020008CE
S315080000B093020008930200089302000893020008BE
S315080000C093020008930200089302000893020008AE
S315080000D0930200089543000893020008930200085B
S315080000E0930200089302000893020008930200088E
S315080000F0930200089302000893020008930200087E
S31508000100930200089302000893020008930200086D
S31508000110930200089302000893020008930200085D
S31508000120930200089302000893020008930200084D
S31508000130930200089302000893020008930200083D
S31508000140930200089302000893020008930200082D
S31508000150930200089302000893020008930200081D
S31508000160930200089302000893020008930200080D
S31508000170930200089302000893020008000000009A
S31508000180930200089302000800F002F800F05CF8F9
S315080001900AA090E8000C82448344AAF10107DA45D4
S315080001A001D100F051F8AFF2090EBAE80F0013F0CA
S315080001B0010F18BFFB1A43F0010318471C4C000037
S315080001C03C4C00000A444FF0000C10F8013B13F0B9
S315080001D0070408BF10F8014B1D1108BF10F8015B92
S315080001E0641E05D010F8016B641E01F8016BF9D185
S315080001F013F0080F1EBF10F8014BAD1C0C1B09D1DC
S315080002006D1E58BF01F801CBFAD505E014F8016B4D
S3150800021001F8016B6D1EF9D59142D6D370470000DF
S315080002200023002400250026103A28BF78C1FBD8F1
S31508000230520728BF30C148BF0B6070471FB504F08E
S31508000240B9FC1FBD10B510BD00F09EF91146FFF7A9
S31508000250F5FF04F061FB00F0BCF903B4FFF7F2FF09
S3150800026003BC04F099FA0000DFF83400016841F491
S3150800027070010160BFF34F8F0A4880470A4800475C
S31508000280FEE7FEE7FEE7FEE7FEE7FEE7FEE7FEE738
S31508000290FEE7FEE705480649044A064B7047000094
S315080002A088ED00E0853F0008890100083024002019
S315080002B0302800203024002072B6704762B6704796
S315080002C072B602B4EFF3118180F31188BFF34F8F32
S315080002D0BFF36F8F084602BC62B6704772B680F3EA
S315080002E01188BFF34F8FBFF36F8F62B6704730BF69
S315080002F0704720BF7047B0FA80F0704790FAA0F0B8
S31508000300B0FA80F0704790FAA0F07047704753EA49
S31508000310020C00F069802DE9F04B4FF00006002B27
S315080003201FBFB3FA83F503FA05F424FA05F65E400F
S3150800033012BF1643B2FA82F502FA05F4C5F1200592
S315080003401EBF22FA05FC44EA0C04203556EA044C82
S315080003504FEA144418BF641C4FF000084FF0000918
S31508000360904271EB030C39D3002919BFB1FA81F712
S3150800037001FA07F6B0FA80F700FA07F6C7F1200780
S315080003801EBF20FA07FC46EA0C062037B6FBF4FC2B
S31508000390A7EB0507103F07F01F0BCBF120060CFA59
S315080003A00BFB2CFA06F644BFB3460026202FA4BF43
S315080003B05E464FF0000B5BEA060C08BF4FF0010BD8
S315080003C019EB0B09ABFB027C48EB0608C01B06FBC6
S315080003D002CC0BFB03CC71EB0C01C1E70B460246C2
S315080003E041464846BDE8F08B13B54FF000004FF084
S315080003F00001AFF30080BDE81C40704740EA0103E6
S31508000400024630B59B0710D14FF0013400E008C210
S3150800041008C91D1B9D4315EAC41FF8D013F0FF0138
S3150800042002F8011B0DD01B0AF8E711F8013B002B57
S3150800043002F8013B05D011F8013B002B02F8013BFD
S31508000440F3D130BD032A40F2308010F0030C00F0DF
S31508000450158011F8013BBCF1020F624498BF11F8F0
S3150800046001CB00F8013B38BF11F8013BA2F10402A9
S3150800047098BF00F801CB38BF00F8013B11F0030321
S3150800048000F05080083AC0F0088051F8043B083A5A
S3150800049051F804CBA0E80810F5E7121D5CBF51F827
S315080004A0043B40F8043BAFF30080D20724BF11F8A1
S315080004B0013B11F801CB48BF11F8012B24BF00F806
S315080004C0013B00F801CB48BF00F8012B70474FF0FD
S315080004D0000200B5134694469646203922BFA0E886
S315080004E00C50A0E80C50B1F12001BFF4F7AF090792
S315080004F028BFA0E80C5048BF0CC05DF804EB890083
S3150800050028BF40F8042B08BF704748BF20F8022BC5
S3150800051011F0804F18BF00F8012B704770477047DD
S315080005207047704710B5203AC0F00B80B1E81850F4
S31508000530203AA0E81850B1E81850A0E81850BFF4BF
S31508000540F5AF5FEA027C24BFB1E81850A0E818505E
S3150800055044BF18C918C0BDE810405FEA827C24BFB2
S3150800056051F8043B40F8043B08BF7047D20728BF40
S3150800057031F8023B48BF11F8012B28BF20F8023B8F
S3150800058048BF00F8012B7047754600F02BF8AE46B9
S3150800059005006946534620F00700854618B020B581
S315080005A0FFF778FEBDE820404FF000064FF0000741
S315080005B04FF000084FF0000B21F00701AC46ACE8FD
S315080005C0C009ACE8C009ACE8C009ACE8C0098D466A
S315080005D0704710B50446AFF300802046BDE81040CA
S315080005E0FFF73BBE00487047D023002072B64EF690
S315080005F02250CEF2000040F2FF01C0F20001017065
S31508000600002080F3098840F67460C2F20000016891
S3150800061081F3088801F03EFF40F6A260C2F20000AE
S3150800062040F6A361C2F200010A78027040F61C7017
S31508000630C2F2000040F62071C2F200010A680260A8
S31508000640106880F30988EFF3148040F0020020F068
S31508000650040080F31488BFF36F8FBDE8F04F0FBC1A
S31508000660BDE8005006BC62B6084726484FF08051E0
S315080006700160704772B640F67862C2F200021168ED
S3150800068081F31188BFF34F8FBFF36F8F62B6EFF315
S3150800069009801EF0100F08BF20ED108A20E9F04FE0
S315080006A040F61C75C2F2000529680860744601F018
S315080006B0F1FE40F6A260C2F2000040F6A361C2F263
S315080006C000010A78027040F62071C2F200010A6839
S315080006D02A6044F0040E1068B0E8F04F1EF0100FC0
S315080006E008BFB0EC108A80F3098840F20002C0F215
S315080006F0000272B682F31188BFF34F8FBFF36F8F74
S3150800070062B6704704ED00E000BFFEE700BFFEE7F3
S3150800071000207047704770B50446A56D00F07CF957
S31508000720064694F83500022808D08020606500BF88
S31508000730002084F8340000BF012070BD20680068DE
S3150800074020F01600216808602068406920F08000C3
S3150800075021684861206C08B9A06C28B12068006837
S3150800076020F00800216808602068006820F0010071
S31508000770216808600FE000F04FF9801B05280AD9A8
S315080007802020606500BF002084F8340000BF0320E5
S3150800079084F83500D1E72068006800F001000028D9
S315080007A0E9D194F85C103F208840A86000BF00207B
S315080007B084F8340000BF012084F835000020BCE727
S315080007C0014691F83500022803D0802048650120AB
S315080007D07047052081F835000868006820F0010098
S315080007E00A6810600020F3E7F8B502460B460025B4
S315080007F0002400200021DEE0012606FA01F51E6825
S3150800080006EA0504AC4275D11E7906F00306012EE8
S3150800081004D01E7906F00306022E13D190684F0005
S315080008200326BE40B0434F00DE68BE4030439060AA
S31508000830506801268E40B0431E79C6F300168E40D6
S31508000840304350601E7906F00306032E09D0D0689F
S315080008504F000326BE40B0434F009E68BE4030435B
S31508000860D0601E7906F00306022E13D1CF0802F1D6
S31508000870200656F827004E07F70E0F26BE40B0434F
S315080008804F07FF0E1E69BE403043CF0802F120060F
S3150800089046F8270010684F000326BE40B0431E796D
S315080008A006F003064F00BE40304310605E6806F04F
S315080008B08056B6F1805F7DD100BF00260096404E77
S315080008C0366846F480463E4F3E603E46366806F435
S315080008D08046009600BF00BF3A4E8F0856F827009C
S315080008E08E07370F0F26BE40B043374EB24202D1AD
S315080008F0002624E05EE0354EB24201D101261EE014
S31508000900334EB24201D1022619E0324EB24201D12B
S31508000910032614E0304EB24201D104260FE02F4ED2
S31508000920B24201D105260AE02D4EB24201D1062671
S3150800093005E02C4EB24201D1072600E008268F07B3
S315080009403F0FBE4030431F4E8F0846F82700264EFD
S315080009503068A0435E6806F48036B6F5803F00D15D
S315080009602043214E3060361D3068A0435E6806F489
S315080009700036B6F5003F00D120431B4E361D3060C9
S31508000980361D3068A0435E6806F48016B6F5801FEB
S3150800099000D12043144E08363060361D3068A04317
S315080009A05E6806F40016B6F5001F00D120430E4E09
S315080009B00C363060491C1029FFF41EAFF8BD000044
S315080009C04438024008380140000002400004024052
S315080009D000080240000C02400010024000140240C9
S315080009E000180240001C0240003C014010B5426954
S315080009F021EA020302EA010443EA0443836110BDC3
S31508000A000AB1816101E00B048361704701480068FF
S31508000A10000C7047002004E0014800687047000099
S31508000A20640E002010B50A48006840F400700849B2
S31508000A3008600846006840F480600860032000F0FB
S31508000A407FF80F2000F006F800F02AF8002010BD05
S31508000A50003C024070B504460E4800784FF47A719F
S31508000A60B1FBF0F00C490968B1FBF0F5284600F037
S31508000A701DFC08B1012070BD102C07D200222146AA
S31508000A80501E00F01EF80548046001E00120F2E758
S31508000A900020F0E76C0E0020700E0020680E002083
S31508000AA0704701460846002809DB00F01F030122AB
S31508000AB09A4043099B0003F1E023C3F8002100BFD5
S31508000AC070472DE9F05F80460D461646002703F06D
S31508000AD047FE074639462A46334601F00700C0F165
S31508000AE0070ABAF1040F02D94FF0040A01E0C0F16F
S31508000AF0070AD14600F1040ABAF1070F02D24FF0ED
S31508000B00000A01E0A0F1030AD4464FF0010A0AFAE6
S31508000B1009FAAAF1010A0AEA020A0AFA0CFA4FF0D5
S31508000B20010B0BFA0CFBABF1010B0BEA030B4AEAC0
S31508000B300B042146404603F01BFEBDE8F09F00006B
S31508000B4000BF00F00702064B19684FF6FF0319406D
S31508000B50044B0B4343EA0221014B196000BF70475F
S31508000B600CED00E00000FA0570B504460D460CB918
S31508000B70012070BD5848006800F00700A84209D255
S31508000B8055490D700846006800F00700A84201D0D4
S31508000B900120EEE7207800F0020002281DD1207817
S31508000BA000F00400042805D14C48006840F4E050E1
S31508000BB04A490860207800F00800082805D1474807
S31508000BC0006840F46040454908604448006820F0E1
S31508000BD0F000A168084341490860207800F0010048
S31508000BE0A8B36068012807D13C4808380068C0F3F4
S31508000BF04040B8B90120BCE76068022802D06068A6
S31508000C00032807D1354808380068C0F3406048B95A
S31508000C100120AEE7314808380068C0F3400008B93B
S31508000C200120A6E72D48006820F003006168084304
S31508000C302A490860FFF7F0FE064609E0FFF7ECFED2
S31508000C40801B41F28831884202D9032091E707E0E8
S31508000C502248006800F00C006168B0EB810FEDD106
S31508000C601D48006800F00700A84209D91A490D7006
S31508000C700846006800F00700A84201D0012078E77E
S31508000C80207800F00400042807D11448006820F4EE
S31508000C90E050E168084311490860207800F0080030
S31508000CA0082808D10D48006820F46040216940EA08
S31508000CB0C1000A49086000F03FF808490968C1F30D
S31508000CC00311074A515CC84006490860064800688F
S31508000CD0FFF7C0FE00204CE7003C024008380240FF
S31508000CE0E44B0008700E0020680E002001480068DA
S31508000CF070470000700E002000B5FFF7F7FF0449A3
S31508000D000968C1F38221034A515CC84000BD00004E
S31508000D1008380240F44B000800B5FFF7E7FF04491E
S31508000D200968C1F34231034A515CC84000BD00005E
S31508000D3008380240F44B00082DE9F0470024002546
S31508000D400026A1462548006800F00C0020B10428BA
S31508000D5005D008283AD105E0DFF8849039E0DFF8B5
S31508000D60849036E01D48001F006800F03F041B48C9
S31508000D70001F006800F4800078B11A481749091F57
S31508000D800968C1F38811A0FB0170014622460023B9
S31508000D903846FFF7BCFA05460EE011480F49091F09
S31508000DA00968C1F38811A0FB017001462246002399
S31508000DB03846FFF7ACFA05460848001F0068C0F336
S31508000DC00140401C4600B5FBF6F902E0DFF810903A
S31508000DD000BF00BF4846BDE8F0870000083802405B
S31508000DE00024F40000127A00F8B504460CB9012074
S31508000DF0F8BD207800F00100002874D0F948006892
S31508000E0000F00C0004280DD0F648006800F00C002D
S31508000E10082813D1F348001F006800F48000B0F5D5
S31508000E20800F0BD1EF4808380068C0F3404000280F
S31508000E3059D06068002856D10120D9E700BF6068FC
S31508000E40B0F5803F08D1E7480838006840F480309C
S31508000E50E449083908601EE06068B0F5A02F0DD196
S31508000E60E0480838006840F48020DE490839086000
S31508000E700846006840F4803008600CE0D948083815
S31508000E80006820F48030D7490839086008460068A9
S31508000E9020F48020086000BF606890B1FFF7BCFDB1
S31508000EA0054606E0FFF7B8FD401B642801D9032074
S31508000EB09EE7CC4808380068C0F340400028F1D0C7
S31508000EC011E0FFF7A9FD054606E0FFF7A5FD401B63
S31508000ED0642801D903208BE7C24808380068C0F3A4
S31508000EE040400028F1D1207800F0020002285FD1A6
S31508000EF0BC48006800F00C0058B1BA48006800F019
S31508000F000C0008281CD1B748001F006800F48000B0
S31508000F10B0B9B44808380068C0F3400020B1E068AA
S31508000F20012801D0012063E7AE480838006820F0A0
S31508000F30F800216940EAC100AA490839086037E083
S31508000F40E06800B30120A8490860FFF765FD05467B
S31508000F5006E0FFF761FD401B022801D9032047E799
S31508000F60A04808380068C0F340000028F1D09D4822
S31508000F700838006820F0F800216940EAC10099495C
S31508000F800839086014E0002097490860FFF744FD17
S31508000F90054606E0FFF740FD401B022801D903205D
S31508000FA026E7904808380068C0F340000028F1D1C9
S31508000FB0207800F0080008282CD16069A8B1012023
S31508000FC08A490860FFF728FD054606E0FFF724FD75
S31508000FD0401B022801D903200AE782486C300068C2
S31508000FE0C0F340000028F1D014E000207F490860D3
S31508000FF0FFF712FD054606E0FFF70EFD401B022827
S3150800100001D90320F4E677486C300068C0F3400045
S315080010100028F1D1207800F00400042870D10027B8
S3150800102070483830006800F0805090B900BF002042
S3150800103000906C483830006840F080506949383173
S3150800104008600846006800F08050009000BF00BFA6
S3150800105001276748006800F48070B0B964480068E2
S3150800106040F4807062490860FFF7D6FC054606E042
S31508001070FFF7D2FC401B022801D90320B8E65C48DA
S31508001080006800F480700028F2D000BFA06801282C
S3150800109008D154486830006840F001005149683169
S315080010A008601DE0A06805280DD14E486830006824
S315080010B040F004004B49683108600846006840F073
S315080010C0010008600CE047486830006820F001001D
S315080010D04449683108600846006820F00400086042
S315080010E000BFA068A8B1FFF797FC054609E0FFF71F
S315080010F093FC401B41F28831884202D9032077E6E7
S3150800110026E0384868300068C0F340000028EED072
S3150800111013E0FFF781FC054608E0FFF77DFC401B5E
S3150800112041F28831884201D9032061E62D486830AA
S315080011300068C0F340000028EFD1012F07D12948E5
S315080011403830006820F0805026493831086000BFE2
S31508001150A069002845D02348006800F00C0008283C
S315080011605DD0A069022845D100201F490866FFF70F
S3150800117053FC054606E0FFF74FFC401B022801D941
S31508001180032035E6174808380068C0F34060002891
S31508001190F1D1D4E907010843616A40EA81110122C5
S315080011A0A06AC2EB500041EA00412C20005D41EAEA
S315080011B000600C49091F086001200B490866FFF703
S315080011C02BFC054606E0FFF727FC401B022801D941
S315080011D003200DE6034808380068C0F3406000287D
S315080011E0F1D049E00838024000004742800E4742E5
S315080011F000700040002021490866FFF70DFC0546EF
S3150800120006E0FFF709FC401B022801D90320EFE599
S315080012101B480068C0F340600028F2D12CE0A069A2
S31508001220012800D1E4E51648001D0668A0690128D2
S3150800123020D006F48001E06981421BD106F03F0107
S31508001240206A814216D147F6C0703040616AB0EB19
S31508001250811F0FD106F440310122A06AC2EB50006B
S31508001260B1EB004F06D106F070612C20005DB1EBA2
S31508001270006F01D00120BBE50020B9E50000474218
S3150800128000380240042808D14FF0E021096941F0EE
S3150800129004014FF0E022116107E04FF0E0210969EF
S315080012A021F004014FF0E0221161704770B5044641
S315080012B02546681EB0F1807F01D301200FE0681E25
S315080012C04FF0E02148610F214FF0FF3003F050FA4C
S315080012D000204FF0E021886107200861002070BDDA
S315080012E07047704701460022002391F83D2091F887
S315080012F03E3042EA030070472DE9F84F044620685D
S3150800130005682068C668206847694FF00009CA461C
S3150800131005F00F09B9F1000F0AD105F0200038B120
S3150800132006F0200020B1204602F06BFEBDE8F88FDB
S31508001330B9F1000F72D007F0010018B906F49070E1
S3150800134000286BD005F0010030B106F4807018B1A2
S31508001350206C40F00100206405F0040030B107F06D
S31508001360010018B1206C40F00200206405F002006C
S3150800137030B107F0010018B1206C40F00400206479
S3150800138005F0080048B106F0200010B907F0010082
S3150800139018B1206C40F008002064206C70B305F08A
S315080013A0200028B106F0200010B1204602F029FEE0
S315080013B020684069C0F3801A206C00F0080010B954
S315080013C0BAF1000F23D0204602F0F0FD20684069EC
S315080013D000F04000402816D12068406920F04000FF
S315080013E021684861A06B50B15648A16B0865A06B8F
S315080013F0FFF7E6F910B1A06B016D88470CE02046AF
S31508001400FFF76FFF08E02046FFF76BFF04E0204672
S31508001410FFF767FF0020206488E7FFE7206B0128B5
S3150800142079D105F01000002875D006F010000028C4
S3150800143071D000BF002000902068006800902068E6
S315080014404068009000BF00BF2068406900F0400077
S31508001450402839D1A06B006840681FFA80F8B8F1B7
S31508001460000F30D0A08D40452DDDA4F82E80A06B4E
S31508001470C069B0F5807F1FD02068C06820F48070EE
S315080014802168C8602068406920F001002168486129
S315080014902068406920F0400021684861202084F8CF
S315080014A03E00002020632068C06820F010002168F4
S315080014B0C860A06BFFF72FF9A08DE28D801A81B264
S315080014C02046FFF70DFF31E7A08DE18D401A1FFA80
S315080014D080F8E08DE8B1B8F1000F1AD02068C0682E
S315080014E020F490702168C8602068406920F00100E7
S315080014F021684861202084F83E0000202063206887
S31508001500C06820F010002168C86041462046FFF7F1
S31508001510E7FE0BE7FFE705F0800030B106F0800034
S3150800152018B1204602F005FF00E705F0400030B18B
S3150800153006F0400018B1204602F053FDF6E600BF5B
S31508001540F4E60000993F000810B504460CB90120DE
S3150800155010BDA06900B100E000BF94F83D0028B9AD
S31508001560002084F83C00204600F028F8242084F85F
S315080015703D002068C06820F400502168C8602046F5
S3150800158002F09EFD2068006920F4904021680861F9
S315080015902068406920F02A00216848612068C068F0
S315080015A040F400502168C86000202064202084F898
S315080015B03D0084F83E000020CAE7000010B586B05A
S315080015C004462D492068884254D100BF00BF002038
S315080015D000902A48006840F010002849086008462C
S315080015E0006800F01000009000BF00BF00BF00BFF9
S315080015F000BF0020009021481438006840F002001F
S315080016001E49143908600846006800F00200009078
S3150800161000BF00BF00BF00BF00BF00200090084603
S31508001620006840F0020008600846006800F0020002
S31508001630009000BF00BF00BF40200190022002902A
S3150800164001200390022004900720059001A90C4868
S31508001650FFF7CAF8802001900720059001A90848DD
S31508001660FFF7C2F82520FFF71CFA032211462520AA
S31508001670FFF727FA06B010BD0010014044380240B3
S315080016800004024070B504460D46164694F83E001E
S31508001690202816D105B10EB9012070BD00BF94F8F7
S315080016A03C00012801D10220F7E7012084F83C001C
S315080016B000BF0020206332462946204602F016FE67
S315080016C0EBE70220E9E700001D4A0168914236D19E
S315080016D01C49098801F4004189BB1A49098801F4A3
S315080016E0804171B1184909780A2903D00021154AA1
S315080016F0118024E01349098841F40041114A1180F8
S315080017001DE0114909780D2906D10E49098841F4C9
S3150800171080410C4A118012E00B490978094A12885F
S31508001720C2F30D02094B995406490988491C054A12
S31508001730118011460988C72901DD002111807047EB
S31508001740001001405C0E00205E0E0020240F0020D1
S31508001750704700BFFEE700BFFEE77047704700000E
S3150800176070B5044600F09EF80020394908703949DA
S315080017700870394908703949086039490860394993
S3150800178008703949087039490870394800680A21CB
S31508001790B0FBF1F0374908603748056845B1374866
S315080017A0066803E0761E002028602D1D002EF9D15C
S315080017B0324801683048006801F0B0FE01F094FA3A
S315080017C001F0B6FA00202E4908602E490880204606
S315080017D001F07CF8208800B170BD204601F082F83F
S315080017E0208800B1F8E700202749086027490880C3
S315080017F0274908602749088027490860274908803B
S31508001800204601F005FE208800B1E5E7204601F0F4
S3150800181025F8208800B1DFE7204601F08BFE2088F6
S3150800182000B1D9E7204601F0BFFC208800B1D3E714
S31508001830204602F041F8208800B1CDE700F0D6FE38
S31508001840FFF78CFF01201649087000BFC4E70000A7
S31508001850800E0020810E0020AE0E00201C0F0020F6
S31508001860200F0020A20E0020A30E0020B40E002098
S31508001870504C0008B00E00201C4C0008204C0008F4
S315080018808C0E0020900E00209C0E0020A00E00203A
S31508001890A80E0020AC0E0020B80E0020BC0E0020BA
S315080018A0820E00200C4909680C4A126801EB820175
S315080018B00B4A11601146096821F0070111600949B0
S315080018C0086800F04041B1F1404F01D000BFFEE783
S315080018D04021054A116070471C4C0008204C00083E
S315080018E0740E002034EF00E0780E002070B5002555
S315080018F038480078012800D070BD00BF4020FEF7A8
S31508001900DFFC054600BF3448007828B900BF2846E2
S31508001910FEF7E4FC00BFEFE72F480078401E2E498B
S3150800192008700846007828B100BF2846FEF7D6FC9E
S3150800193000BFE1E72948007828B100BF2846FEF72E
S31508001940CDFC00BFD8E7264801682648006801F0A4
S31508001950D1FD0446012C02D0002000F0ABF901F0BD
S31508001960B9F9214908700846007800EB40001F497C
S3150800197051F820001E490860084600681D49096894
S3150800198088420FD1002000F069FD0446012C03D0DF
S315080019901848006800F08EF900BF2846FEF79EFC3E
S315080019A000BFA9E712480068D0F89400401C104907
S315080019B00968C1F8940010480068401C0E49086080
S315080019C0FEF753FE00BF2846FEF788FC00BF00BF9F
S315080019D092E70000810E0020800E0020AE0E002047
S315080019E0204C00081C4C0008A30E00207420002080
S315080019F0200F00201C0F0020DC0E00202DE9F041EE
S31508001A0004460E46154600272148007820B142F6BE
S31508001A10E1602880BDE8F0811CB945F6C3502880EE
S31508001A20F8E700BF00BF4020FEF74AFC074600BFA4
S31508001A3000BF1849206888420AD100BF00BF38464F
S31508001A40FEF74CFC00BF00BF45F6C1502880E1E711
S31508001A5010482060666000202062606284F82800D2
S31508001A60E06204F1080001F080F8204600F0A0FFCB
S31508001A7009480088401C0849088000BF00BF38464E
S31508001A80FEF72CFC00BF00BF0020288000BFC1E77E
S31508001A90800E00204D555458A00E00202DE9F04721
S31508001AA00646894617461C46089D4FF0000A7C489C
S31508001AB0007820B146F2AE102880BDE8F087794854
S31508001AC00078012803D045F689602880F5E71EB915
S31508001AD045F6C3502880F0E71FB1B7F5004F02D18D
S31508001AE000E000BF03E045F625602880E5E700BF73
S31508001AF06D493068884203D045F6C4502880DCE733
S31508001B0000BF00BF4020FEF7DBFB824600BF00BFD8
S31508001B1096F82800B8B9654800687062012086F80A
S31508001B2028000CB1F06A206031466048006800F071
S31508001B3057FF00BF00BF5046FEF7D0FB00BF00BFEF
S31508001B4000202880B9E75949706A0968884221D176
S31508001B5096F82800FF280AD100BF00BF5046FEF7B6
S31508001B60BDFB00BF00BF45F284702880A5E796F844
S31508001B702800401C86F828000CB1F06A206000BFD7
S31508001B8000BF5046FEF7AAFB00BF00BF45F28270B1
S31508001B90288092E707F4004068B100BF00BF5046AE
S31508001BA0FEF79CFB00BF00BF0CB10020206046F288
S31508001BB0B010288081E73E48007868B100BF00BFB2
S31508001BC05046FEF78BFB00BF00BF0CB1002020601B
S31508001BD046F66350288070E7D6F8248098F83B00CC
S31508001BE03249096891F83B10884206DD2F4800689B
S31508001BF090F83B10404601F05DFB4B4604222B480B
S31508001C000168304600F042FF00BF00BF5046FEF7AD
S31508001C1065FB00BF00BF00F055F800BF00BF4020BD
S31508001C20FEF74EFB824600BF00BF2048006890F8CA
S31508001C30390030B101280CD002281AD0032821D146
S31508001C4010E01CB119480068C06C2060002028808C
S31508001C501CE01CB115480068C06C206046F2A9104B
S31508001C60288013E00CB10020206047F2D920288094
S31508001C700CE01CB10D480068C06C206045F6C250E7
S31508001C80288003E046F62E60288000BF00BF00BF0C
S31508001C9000BF5046FEF722FB00BF00BF00BF0CE79F
S31508001CA0800E0020810E00204D5554581C0F002030
S31508001CB0AE0E002010B5044600BFFEF727FD00BF94
S31508001CC010BD000010B5002422480078012800D075
S31508001CD010BD2148007800B1FAE72048007800B125
S31508001CE0F6E700BF4020FEF7EBFA044600BF00F017
S31508001CF0F1FF1B4908700846007800EB40001949B7
S31508001D0051F820001849086008460068174909680C
S31508001D10884205D100BF2046FEF7E0FA00BFD7E7A4
S31508001D2011480068D0F89400401C0F490968C1F8AA
S31508001D3094000F480068401C0D490860FEF795FCA2
S31508001D4000BF2046FEF7CAFA00BFBFF36F8F00BF79
S31508001D50BEE70000810E0020800E0020AE0E002097
S31508001D60A30E002074200020200F00201C0F002046
S31508001D70DC0E002070B504461C480078012803D004
S31508001D8045F68B60208070BD00256D1C6D1C6D1C92
S31508001D9017480088A84203DC45F68C602080F2E7E5
S31508001DA014480078E8B900F095FF1349087008460A
S31508001DB00078124908701048007800EB4000104976
S31508001DC051F820000F490860084600680E49086067
S31508001DD0012008490870FEF709FC43F6992020807F
S31508001DE002E045F68A60208000BFCCE7820E00201C
S31508001DF0E40E0020810E0020A30E0020A20E002073
S31508001E0074200020200F00201C0F00202DE9F0412F
S31508001E1007464FF0000800BF00BF4020FEF750FA03
S31508001E20804600BF00BF00203B4908803B49086048
S31508001E303B4908603B4908603B4908603B490860E4
S31508001E403B49088100BF00BF4046FEF747FA00BF7E
S31508001E5000BF00BF00BF4020FEF732FA804600BF31
S31508001E6000BF3448046800BF00BF4046FEF736FA94
S31508001E7000BF00BF21E000BF00BF4020FEF720FAE8
S31508001E80804600BF00BF002044F8800FE062606112
S31508001E902082608220626062FEF73AFCE061803C44
S31508001EA004F16C060020B081D4F8BC4000BF00BF26
S31508001EB04046FEF713FA00BF00BF002CDBD100BF77
S31508001EC000BF4020FEF7FCF9804600BF00BF1A4855
S31508001ED0056800BF00BF4046FEF700FA00BF00BF16
S31508001EE013E000BF00BF4020FEF7EAF9804600BFB6
S31508001EF000BF05F120060020B081AD6900BF00BF14
S31508001F004046FEF7EBF900BF00BF002DE9D10020DF
S31508001F103880BDE8F0810000C20E0020D80E0020EF
S31508001F20F40E0020F80E00200C0F0020100F0020E1
S31508001F3068200020E00E0020A80E00207047000050
S31508001F402DE9FF4F85B004469346DDE91995DDE98D
S31508001F501286159F002002906248007828B147F241
S31508001F604A10288009B0BDE8F08F1CB947F2AD10B9
S31508001F702880F7E7BBF1000F03D147F24F102880FE
S31508001F80F0E71EB946F62F602880EBE7564800684A
S31508001F90874203D246F630602880E3E71498B842B1
S31508001FA003D346F631602880DCE7B8F11E0F06D960
S31508001FB0B8F11F0F03D046F273202880D2E7B8F194
S31508001FC01F0F06D14948844203D046F27320288061
S31508001FD0C8E7204601F02CFA0020288009F0010005
S31508001FE010B909F0020088B109F0020070B1B246D2
S31508001FF00020049007E00020CAF800000AF1040A4D
S315080020000498401C04900498B842F4D3149806EB3C
S3150800201080000390CDE9007932465846039B08991B
S3150800202000F0B4F98246B24503D246F632602880FB
S3150800203098E73946304601F071FAC4F824B0089892
S31508002040A0620698E06084F83B8084F83C80C4F877
S3150800205000A00398A0601798E065179818B9244857
S315080020600068206601E01798206618986060266266
S315080020706764A4F8489004F16C00169900F090FC87
S31508002080204600F03BF800BF00BF4020FEF718F9D5
S31508002090029000BF00BF94F83B0000F031FE2046D6
S315080020A000F08EFE204601F079F912480088401C9F
S315080020B01049088010480078012807D000BF00BFE3
S315080020C00298FEF70BF900BF00BF4BE700BF00BF41
S315080020D00298FEF703F900BF00BFFFF7F3FD00BF44
S315080020E040E70000800E00204C4C0008A41F00208A
S315080020F0B00E0020E40E0020810E0020704700007C
S315080021002DE9F04104460E464FF000086148007874
S3150800211020B147F24E103080BDE8F0815E48007865
S31508002120012803D045F689603080F5E75B4884428C
S3150800213003D147F24C103080EEE784B900BF00BFE8
S315080021404020FEF7BDF8804600BF00BF544804682B
S3150800215000BF00BF4046FEF7C1F800BF00BF00BF82
S3150800216000BF4020FEF7ACF8804600BF00BF94F8D9
S315080021703A0008285ED2DFE800F004090E10080AC3
S315080021800F11204600F03AFE5FE05EE000BF2046F1
S3150800219001F07AFA59E000BF00BF00BF94F8380092
S315080021A0082839D2DFE800F0040705380D080906C3
S315080021B000BF00BF31E000BF00BF204600F00DFDA4
S315080021C02BE0606B456A15F83B7F204600F005FD5D
S315080021D0287869783B3D884212D095F83B0094F8F8
S315080021E03B1088420CD1284600F02DFC074695F88E
S315080021F03C00B84202DA95F83C0000E0384607464B
S31508002200002084F8380095F83B00B84203D03946D8
S31508002210284601F04FF800E000BF00BF94F83A00E6
S31508002220032803D094F83A00072802D1204601F083
S315080022302BFA0AE000BF00BF4046FEF74FF800BF82
S3150800224000BF46F62D60308066E700BF206C10B1EF
S31508002250204600F0C9FB04F16C0000F081FB204623
S3150800226000F022F8204601F0B1F80E480088401E1A
S315080022700C490880FF2084F83A000020308000BF0F
S3150800228000BF4046FEF72AF800BF00BFFFF71AFD59
S3150800229000BF41E7800E0020810E0020A41F002009
S315080022A01C0F0020E40E0020704770472DE9F05FF0
S315080022B005460E4617461C464FF0000B3148007877
S315080022C020B147F259102080BDE8F09F1EB946F2AA
S315080022D0D5202080F8E71FB946F2D5202080F3E7FD
S315080022E000BF00BF4020FDF7EBFF834600BF00BFDD
S315080022F00DB925480568286868B900BF00BF584663
S31508002300FDF7ECFF00BF00BF00203060386047F2E1
S3150800231052102080D8E795F8480000F0010068B907
S3150800232000BF00BF5846FDF7D9FF00BF00BF002019
S315080023303060386047F254102080C5E7D5F820A0F1
S315080023400AF1200AD5F8449000BF00BF5846FDF7A9
S31508002350C5FF00BF00BF4FF0000803E00AF1040AFA
S3150800236008F10108C84503D2DAF800000028F5D0BC
S31508002370C6F80080A9EB080038600020208000BF5E
S31508002380A2E70000800E00201C0F0020F0B50446CE
S31508002390DDE9055602EB850020F007004FF0807C4A
S315080023A0071F3846C7F800C0071F38463C60DFF8E5
S315080023B0A8C0071F3846C7F800C04FF0123C071FD1
S315080023C03846C7F800C04FF0033C071F3846C7F821
S315080023D000C04FF0023C071F3846C7F800C0071F69
S315080023E038463B60071F384639606FF0020C071FF6
S315080023F03846C7F800C04FF0113C071F3846C7F8E3
S3150800240000C04FF0103C071F3846C7F800C04FF011
S31508002410093C071F3846C7F800C04FF0083C071F9D
S315080024203846C7F800C04FF0073C071F3846C7F8BC
S3150800243000C04FF0063C071F3846C7F800C04FF0EB
S31508002440053C071F3846C7F800C04FF0043C071F75
S315080024503846C7F800C0F0BDDD34000830B504467C
S315080024600CB90B480468216A2068884206D3616C57
S31508002470206A00EB81002168884201D8002030BD1F
S31508002480616C206A01F036F805462846F7E7000031
S315080024901C0F002070B5FEF73BF905461548006885
S315080024A015490968884215D012480068D0F89C007A
S315080024B0281A10490968C1F898000E480068D0F82B
S315080024C0A0000C490968D1F8981008440949096818
S315080024D0C1F8A00008480068C0F89C500020FFF723
S315080024E0BDFF0446012C03D002480068FFF7E2FB53
S315080024F070BD00001C0F0020200F00202DE9F041C0
S3150800250006460D46144600272748007820B147F2AC
S3150800251075202080BDE8F08124480078012803D082
S3150800252045F689602080F5E72148007818B146F617
S3150800253063502080EEE735B1022D05D0042D05D075
S31508002540082D04D101E000BF00BF00BF03E045F637
S3150800255025602080DEE700BF00BF00BF4020FDF7F2
S31508002560AFFE074600BF00BF23462A46314611483C
S31508002570006801F043F8208838B100BF00BF38462C
S31508002580FDF7ACFE00BF00BFC4E70A48006800F0CC
S3150800259035FC00BF00BF3846FDF7A0FE00BF00BFF0
S315080025A0FFF790FB00BFB5E7800E0020810E0020E4
S315080025B0AE0E00201C0F002070B50446002600BF92
S315080025C000BF4020FDF77CFE064600BF00BF064858
S315080025D0056800BF00BF3046FDF780FE00BF00BF9C
S315080025E000202080284670BDE80E00200EB547481A
S315080025F0029047480090474802904748029047484B
S31508002600009047480290474801904748029047483B
S315080026100290474802904748029047480190474829
S31508002620019047480190474802904748019047481B
S31508002630029047480190474801904748019047480B
S3150800264001904748029047480290474802904748F9
S3150800265001904748029047480290474801904748EA
S3150800266001904748019047480190474801904748DC
S3150800267001904748029047480290474802904748C9
S3150800268002904748019047480190474801904748BB
S3150800269002904748029047480290474801904748A9
S315080026A0019047480190474800904748019047489D
S315080026B00290474802904748029047480290474888
S315080026C00290474802904748029047480190474879
S315080026D0029047480290474801904748019047486A
S315080026E0029047480290474801904748019047485A
S315080026F0029047480290474801904748019002983F
S31508002700029001980190009800900EBD704C000848
S31508002710D44D0008714C0008724C0008744C00082F
S31508002720784C00087C4C0008794C0008A44C00083A
S31508002730A54C0008A64C0008A84C0008AA4C00089E
S31508002740AC4C0008CC4C0008CE4C0008D04C000815
S31508002750D24C0008D44C0008D64C0008D84C0008C7
S31508002760084D0008094D00080A4D00080C4D0008E0
S315080027700E4D00080F4D0008104D0008124D0008B8
S31508002780144D0008164D0008184D00081C4D000889
S315080027904C4D00084D4D00084E4D00084F4D0008A1
S315080027A0504D0008524D0008544D00087C4D000855
S315080027B07D4D00087E4D00087F4D0008804D0008BD
S315080027C0824D0008844D0008884D0008894D000890
S315080027D08A4D00088B4D00088C4D00088D4D000869
S315080027E08E4D00088F4D0008904D0008924D000848
S315080027F0934D0008944D0008964D0008984D000822
S31508002800994D00089A4D00089C4D0008CC4D0008CB
S31508002810CD4D0008CE4D0008D04D0008002400BF5D
S3150800282000BF00BF4020FDF74BFD044600BF00BFB8
S3150800283008480068401C0749086007480068401CAB
S315080028400549086000BF00BF2046FDF747FD00BFE9
S31508002850E6E700007C0E0020C40E002010B58AB002
S31508002860044600200E4908600B2000210591CDE999
S315080028700704069108460B4909680B4A12680B4B70
S315080028801B68CDE90132CDE903101F200023084A51
S3150800289008A100900C48FFF753FB0AB010BD0000D2
S315080028A07C0E0020144C0008104C00080C4C000844
S315080028B01D28000875432F4F532D4949492049645F
S315080028C06C65205461736B00A41F00200021034A25
S315080028D01160034A1180018070470000940E0020A1
S315080028E0980E002070B501461A4D2D681DB945F29F
S315080028F01E750D8070BD184D2D881DB945F21D75C4
S315080029000D80F7E7134D28682A681032124D2D8876
S315080029106D1EACB2002308E0026000254560058103
S31508002920C560103010325D1CABB2A342F4DB002543
S31508002930056045600581C560064D2D68074E356002
S31508002940054D2D88B5800025F58035810D8000BFA1
S31508002950D0E70000304C0008284C0008682000200A
S3150800296010B5014648894B89BBB10A680B4B1B68F1
S3150800297013600A4C4B6823602346DB884C891B1B73
S31508002980064CE38023469B884C892344034CA3804A
S3150800299000234B818B810B604B6010BD68200020A3
S315080029A001810022428182810260426070470000F4
S315080029B009A1C161002141610849096811B90021CD
S315080029C0816105E00549096881610449096848612A
S315080029D00249086070470000200000009C0E002095
S315080029E0026C0A62016470472DE9F84305462C6CAF
S315080029F025E0D4F82090FDF78BFE8046C4F82C809D
S31508002A002146284600F034F804F10806306820B953
S31508002A10002084F82800606210E0376865620120AB
S31508002A2084F8280021463846FFF7DAFF00231A46BD
S31508002A3039462046CDF8008000F0F6F84C46002CC2
S31508002A40D7D1BDE8F88330B504461F2004F140010C
S31508002A500AE00D68AB6823B193F83B20824200DA9E
S31508002A6010460D6805F120010D68002DF1D130BD25
S31508002A70024602F1400002E0036803F12000036801
S31508002A808B42F9D103681B6A036070472DE9F04150
S31508002A9005460C4616461F4684F83860002084F81A
S31508002AA039003946204600F0EDFB3DB105F108082E
S31508002AB065632146404600F05DF801E0002060634A
S31508002AC02146284600F002F8BDE8F08110B540B16D
S31508002AD04468C1F8C04000F108031A68D468C461A4
S31508002AE013E091F83840022C02D0072C08D103E0F5
S31508002AF006A4C1F8C04007E006A4C1F8C04003E038
S31508002B0007A4C1F8C04000BF00BF10BD5461736B75
S31508002B10205100005461736B2053656D000000005E
S31508002B202000000010B50A4606A4C2F8C04040B10D
S31508002B3000F10803196811B1CC68C46101E001A469
S31508002B40C46110BD2000000070B50446666B06F12E
S31508002B5008052868C06A38B1204600F03EF8666362
S31508002B602146284600F006F870BD00210160416044
S31508002B700181704710B591F83B3004683CB90124CF
S31508002B8004810024CC620C630160416024E004895E
S31508002B90641C0481026805E092F83B409C4200DD13
S31508002BA002E0D26A002AF7D100BF3AB90024CC6203
S31508002BB044680C630C6BE16241600DE0146B2CB940
S31508002BC0CA6200240C631163016005E0CA62146BD3
S31508002BD00C630C6BE162116310BD10B5446B14B342
S31508002BE0446B04F108010C68E46A1CB900240C6003
S31508002BF04C6011E0046B24B9C26A002414630A60AD
S31508002C000AE0C46A24B9036B0024DC624B6003E063
S31508002C10036BC26ADA6213630C89641E0C81002492
S31508002C20C4620463446310BD2DE9F04105460C46B1
S31508002C3016461F46DDF8188094F83A00082845D24B
S31508002C40DFE800F0040508090607272800BF00BFCB
S31508002C5000BF3CE000BF6666A4F86870C4F84C8004
S31508002C6015B12046FFF7B9FF21462846FFF75AFF58
S31508002C7094F83A00032802D1204600F005FD2046C4
S31508002C8000F068F800203834A070607004F838093D
S31508002C901DE000BF6666A4F86870C4F84C8015B1DC
S31508002CA02046FFF79AFF21462846FFF73BFF94F890
S31508002CB03A00072802D1204600F0E6FC0420383402
S31508002CC0A0700020607004F8380900E000BF00BF5B
S31508002CD0BDE8F08110B503490868FDF70CFBC0B2E2
S31508002CE010BD0000A40E0020002004E00021034AC5
S31508002CF042F82010401C0028F8D07047A40E002087
S31508002D0004490968C0F11F0301229A401143014A88
S31508002D1011607047A40E002004490968C0F11F031A
S31508002D2001229A409143014A11607047A40E00207F
S31508002D30002109E001EB4102054B03EB820000226A
S31508002D40028102604260491C2029F3D370470000C3
S31508002D507420002010B5044694F83B00FFF7D0FF16
S31508002D6094F83B0005490978884203D1204600F0CB
S31508002D7027F802E0204600F003F810BDA20E002056
S31508002D8010B590F83B3003EB43030C4C04EB83017E
S31508002D900B683BB901230B8100230361436108607B
S31508002DA0486009E00B895B1C0B810B6803610023F3
S31508002DB043610A685061086010BD00007420002055
S31508002DC010B590F83B3003EB43030B4C04EB83013F
S31508002DD00B683BB901230B8100230361436108603B
S31508002DE0486008E00B895B1C0B81002303614A6875
S31508002DF042611061486010BD742000202DE9F04141
S31508002E00054695F83B0000EB4000124901EB8004AB
S31508002E106F692E6987B946B90020208120606060F5
S31508002E2095F83B00FFF778FF0EE02089401E2081C9
S31508002E3000207061266007E02089401E20813E61DF
S31508002E400EB9676000E07761002068612861BDE817
S31508002E50F08100007420002088B00020009006E071
S31508002E60BD490968480002AA0021FFF747FBBB488D
S31508002E7000780128F4D102A8FEF7C8FF4FF0000831
S31508002E80B7480068B4490968884205D9B448006853
S31508002E90B1490968B0FBF1F8B8F1000F04D1B048A0
S31508002EA000680A21B0FBF1F800BFFDF731FC814646
S31508002EB000BF00BF4020FDF703FA009000BF00BF27
S31508002EC0A8480068A84908600020A649086000BF0D
S31508002ED000BF0098FDF702FA00BF00BFA3480068CC
S31508002EE0A1490968884248D9A0480068A04988428B
S31508002EF005D242F2107004900120039023E09B480B
S31508002F0000689C49884205D24FF47A7004900A20DA
S31508002F10039018E0954800689749884203D26420D0
S31508002F20049003900FE0914800689449884205D2BE
S31508002F300A2004904FF47A70039004E0012004906C
S31508002F4042F210700390894801680398B1FBF0FBC0
S31508002F508549049809684843B0FBFBF042F21071B2
S31508002F60081A87490880874800880988884207DA46
S31508002F70834800888349088002E000208049088049
S31508002F80FEF7DCFF002500BF00BF4020FDF798F9DB
S31508002F90009000BF00BF7C48046800BF00BF0098CF
S31508002FA0FDF79CF900BF00BF28E000BF00BF402026
S31508002FB0FDF786F9009000BF00BF54F8A00F6060C7
S31508002FC0002044F8A00900BF00BF0098FDF786F965
S31508002FD000BF00BFD4F8A400054400BF00BF4020CE
S31508002FE0FDF76EF9009000BF00BFD4F8BC4000BFE3
S31508002FF000BF0098FDF772F900BF00BF002CD4D1BE
S315080030005DB35B48854205D242F2107006900120F6
S3150800301007901DE05748854205D24FF47A7006900E
S315080030200A20079014E05448854203D2642006908B
S3150800303007900DE05148854205D20A2006904FF4C4
S315080030407A70079004E00120069042F2107007900B
S315080030500798B5FBF0F0059003E0002006900120E4
S31508003060059000BF00BF4020FDF72AF9009000BF79
S3150800307000BF4548046800BF00BF0098FDF72EF959
S3150800308000BF00BF2CE0D4F8A40006994843059970
S31508003090B0FBF1F086B242F21070864200D90646BD
S315080030A0A4F89060B4F89200B04201DAA4F89260ED
S315080030B002AB04F1B002111D2046FFF7F7F800BF76
S315080030C000BF4020FDF7FCF8009000BF00BFD4F811
S315080030D0BC4000BF00BF0098FDF700F900BF00BF65
S315080030E0002CD0D100272948D0F800A00AF1200AE0
S315080030F0274800680838019002E00AF1040A7F1C94
S31508003100DAF8000010B901988742F6D3214807601B
S315080031101F480068C01B204908602048007801281D
S3150800312005D100201D49087002A8FEF76FFEFDF7BD
S31508003130EFFAA0EB09001A4908601A4800680968FE
S31508003140884203D2164800681649086002AA002178
S315080031504046FFF7D3F9A8E6384C0008D00E002001
S31508003160504C0008C40E0020CC0E0020C80E0020CB
S31508003170801A060000093D00005A62020084D7172B
S31508003180C00E0020C20E0020E00E00201C4C0008D5
S31508003190204C0008840E0020880E0020BE0E002059
S315080031A0D40E0020D80E002010B58AB004460020A0
S315080031B021490860214908602149086021490870A9
S315080031C0214908702149086021490860214800689A
S315080031D020B946F62B6020800AB010BD1E4800684C
S315080031E01E490968884203D246F62C602080F3E718
S315080031F01B4800781F2803D346F62A602080EBE791
S31508003200032000210591CDE90704069108461249D5
S315080032100A68144909680F4B1B68CDE90131CDE9E5
S3150800322003200F48007800230F4A10A10090144885
S31508003230FEF786FE00BFCFE7C40E0020CC0E0020A6
S31508003240C80E0020D00E0020BE0E0020840E0020DE
S31508003250880E00203C4C0008444C00084C4C0008E2
S31508003260344C0008404C0008592E000875432F4F6F
S31508003270532D4949492053746174205461736B0076
S31508003280F421002070B504460D4655B12B46084872
S3150800329000210268204600F05BF9032084F83A0012
S315080032A002E0022084F83A002046FFF7A7FD70BD29
S315080032B0E80E00202DE9F04104460D4600BF002621
S315080032C094F83B7094F83A0008285DD2DFE800F0DD
S315080032D004191E1F1A1B20212046FFF78FFD84F8AC
S315080032E03B5094F83B00FFF70BFD2B4800688442DF
S315080032F003D12046FFF744FD02E02046FFF760FDB4
S3150800330044E000BF00BF84F83B503FE000BF00BF69
S3150800331000BF84F83B5094F8380008282FD2DFE81D
S3150800332000F02E042F2E0A05063000BF00BF2046E7
S31508003330FFF70AFC26E02046FFF706FC606B466AA4
S31508003340AF4205DD96F83B00A84217DC002615E0DB
S3150800335096F83B00B84211D13046FFF774FB054694
S3150800336096F83C00A84202DA96F83C0000E02846A7
S31508003370054696F83B00A84200D1002602E000BFA9
S3150800338000BF00BF00BF01E0BDE8F08100BF3446C2
S31508003390002C94D100BFF7E71C0F00200021C0F8CD
S315080033A0B8100949096819B90021C0F8BC1007E026
S315080033B005490968C0F8BC1003490968C1F8B8008E
S315080033C00149086070470000E00E0020D0F8B820D8
S315080033D0D0F8BC104AB90D4B196011B10023C1F8D9
S315080033E0B8300023C0F8BC300FE029B90023C2F872
S315080033F0BC30C0F8B83008E0C2F8BC10C1F8B82034
S315080034000023C0F8BC30C0F8B8307047E00E002082
S315080034100021044A1160044A1180044A116001809F
S3150800342070470000E00E0020E40E0020DC0E0020AD
S3150800343010B5044600202060A060606020616061CD
S31508003440A061E06122A0E060002020626062A062C4
S31508003450E0646066A4F86800002104F16C00FFF7D8
S315080034609FFA00202C3420656065A065A4F86000EA
S31508003470E0656062E067C4F88000A06184F86200D5
S31508003480C4F88800C4F88400A083A062E0622063C0
S315080034906063A4F86400A4F86600A066E066FDF719
S315080034A037F920670020606720606060A06020739D
S315080034B06073A0732020E073207400206061C4F854
S315080034C08C00C4F8900004A0C4F894002C3C10BDED
S315080034D03F5461736B0000002000000008B50448E3
S315080034E00068FEF7E2FE69460020FEF709FE08BD01
S315080034F01C0F002010B502460B46002107E0064CBB
S315080035001068A04201D0002010BD121D491C0829D0
S31508003510F5D30120F8E700004523CDAB024600208D
S3150800352003E0034B42F82030401C0828F9D37047C3
S315080035304523CDAB00210180034A1160034A11607F
S315080035409180D18070470000E80E0020EC0E002024
S315080035502DE9F04304460F469446984608EB0C00BE
S31508003560DFF89090D9F80090B944A0EB09021AB98F
S3150800357000206065BDE8F0831F4B186838B962659E
S315080035800020A061E0611C6001209880F2E798881D
S31508003590401C98801968486DC61BB2420BD2C86990
S315080035A048B96265B01A48650020E061A161CC613E
S315080035B01C600120DEE7921B0D46A96903E0486DF1
S315080035C0121A0D46896911B1486D9042F7D949B169
S315080035D0CD696265E561A161486D801A4865CC616F
S315080035E0AC6104E06265E5610020A061AC61012080
S315080035F0C0E70000E80E0020EC0E00202DE9F04F91
S3150800360006460C4691461F464FF0000BB9F1040FCB
S3150800361001D1002520E0B9F1080F1BD124B947F2E2
S315080036207E203880BDE8F08FB56D16480068A0EB9F
S315080036300508A0450AD3B8FBF4F004FB0055B8FB0F
S31508003640F4F004FB108000B12544B565B06D204444
S31508003650B06501E00B48056823462A4659463046B8
S31508003660FFF776FF8246BAF1010F05D1012086F8E9
S315080036703A000020388002E047F27E20388000BFFA
S31508003680D0E70000E80E002030B5C3698169134A07
S315080036909BB921B900241460948044651CE0002479
S315080036A0CC614C6D456D2C444C6511609488641E44
S315080036B094800024846144650EE0996121B1CB6150
S315080036C04C6D456D2C444C650024C4619488641E79
S315080036D0948000248461446530BD0000EC0E00200F
S315080036E010B5002400BF00BF4020FCF7E9FD0446E2
S315080036F000BF00BF0848094908600948086201F187
S315080037000800FFF732FA00BF00BF2046FCF7E6FDC7
S3150800371000BF00BF10BD0000434F4E44B822002032
S31508003720DC220020F8B5002600BF00BF4020FCF7C9
S31508003730C7FD064600BF00BFFCF7EAFF04460F4870
S31508003740C4620F4D286838B900BF00BF3046FCF781
S31508003750C5FD00BF00BFF8BD00231A460949084841
S3150800376008380094FFF760FA00BF00BF3046FCF740
S31508003770B5FD00BF00BF00BFEDE70000DC2200205A
S31508003780C02200200C2300202DE9F84307464FF0FD
S31508003790000800BF00BF4020FCF792FD804600BF2E
S315080037A000BFFCF7B5FF06463F48C66201463F48DC
S315080037B0FFF75EF93C4D08353C4890F83B003B491D
S315080037C091F83C1088420AD0384890F83C003749AE
S315080037D081F83B00084690F83C003549087028688F
S315080037E028B900203049486281F8280010E02C6882
S315080037F02D48446201202C4981F828002046FFF70D
S31508003800EFF800231A46214627480096FFF70CFAD8
S315080038103B46032225492748FFF738F900BF00BF72
S315080038204046FCF75BFD00BF00BFFEF74BFA00BF42
S3150800383000BF4020FCF744FD804600BF00BF1A4881
S31508003840406A80B918491948FFF7CAF8174816494F
S315080038504862012081F8280000BF00BF4046FCF7F7
S315080038603DFD00BF1DE01048446A94F83B000F492F
S3150800387091F83B10884205DD0C4890F83B1020462D
S31508003880FFF718FD0023042208490748FFF7FEF84A
S3150800389000BF00BF4046FCF721FD00BF00BFFEF792
S315080038A011FABDE8F8830000DC2200200C23002072
S315080038B0A20E0020B822002010B58AB004460020C7
S315080038C02A4908802A4908602A4908602A4908803E
S315080038D02A4800682A490968B0FBF1F029490860B6
S315080038E000202949086029490860224628A12C4851
S315080038F0FEF784F8208808B10AB010BDFFF7F0FE7D
S315080039002848006818B947F247302080F4E7264867
S31508003910006826490968884203D247F24830208061
S31508003920EAE7234800781F2803D347F24630208069
S31508003930E2E70B20002105910A46CDE90704069126
S31508003940194800681B490968164B1B68CDE90131FF
S31508003950CDE90302164800780023174A17A10090FC
S315080039601C48FEF7EDFA00BFC6E70000080F002066
S31508003970FC0E0020040F0020000F0020504C000809
S31508003980584C0008180F00200C0F0020100F0020BC
S315080039904F5320546D72204D7574657800000000F1
S315080039A0DC2200205C4C0008644C00084C4C0008E3
S315080039B0544C0008604C0008A93A000875432F4F7C
S315080039C0532D4949492054696D6572205461736BBA
S315080039D0000000000C2300202DE9F0470546884624
S315080039E02848006870B90020286168612548056084
S315080039F00120254908802548C0F80080FFF792FE77
S31508003A00BDE8F08720480088401C1F490880A8693F
S31508003A1040441E490968461A1A480468D4F818909A
S31508003A204E4510D2606970B9A9EB0600A061002066
S31508003A3068612C616561134805601448C0F8008008
S31508003A40FFF770FEDCE7A6EB090627463C6903E0AC
S31508003A50A069361A2746246914B1A069B042F7D975
S31508003A604CB16769AE616F612C61A069801BA0616A
S31508003A7065613D6104E0AE616F61002028613D61CA
S31508003A8000BFBDE7040F0020000F0020140F002020
S31508003A901CB501A800231A46194600900148FDF7EF
S31508003AA0FDFF1CBDDC2200204FF0000AFFF7F0FFE7
S31508003AB000BF3D48006810B94FF0000903E03A48D6
S31508003AC00068D0F818904846FFF75EFE364800684A
S31508003AD000B9EEE7FCF71CFE804600BF00BF402099
S31508003AE0FCF7EEFB824600BF00BF3048076800BF00
S31508003AF000BF5046FCF7F2FB00BF00BF2C48006829
S31508003B003D1A2B480760284804680CE0A069A842BB
S31508003B1004D2A0692D1A0020A06103E0A069401B09
S31508003B20A061002524690DB1002CEFD11E48046858
S31508003B3026E0042084F82600A66816B12046E16827
S31508003B40B04794F82600042818D119480168204679
S31508003B5000F034F8A08C022809D184F82600206ADF
S31508003B60A061134801682046FFF736FF06E00020EB
S31508003B7060612061A061032084F826000A48046871
S31508003B8014B1A0690028D4D0FCF7C2FDA0EB080048
S31508003B9008490860084800680968884203D2054849
S31508003BA000680549086084E7040F0020E80E002035
S31508003BB0140F00200C0F0020100F00202DE9F041F3
S31508003BC005460F46D5F814802C69B8F1000F40D188
S31508003BD054B900202949086029490880A86129485C
S31508003BE00760FFF79FFD46E025480088401E2449E8
S31508003BF00880244800683E1A00206061A069A96907
S31508003C000844A0611D4804600EE0A069B04204D2D1
S31508003C10A069361A0020A06103E0A069801BA06194
S31508003C200026A046D8F810400EB1002CEDD1134856
S31508003C3000688069A969884203D1104800688069CC
S31508003C4018B910480760FFF76DFD00202861A861C4
S31508003C5011E00B480088401E09490880C8F8104042
S31508003C602CB1C4F81480A069A9690844A061002091
S31508003C7068612861A861BDE8F0810000040F002092
S31508003C80000F0020140F00202DE9F04104460D46D0
S31508003C9016460E4F00BF387808B900F0A5FB00BFDE
S31508003CA0EFF311800746202080F3118800BF00BF7C
S31508003CB032462946204600F00BF88046F8B280F3D3
S31508003CC0118800BF00BF4046BDE8F0818C12002075
S31508003CD02DE9F047074688461646C24607EB4701D0
S31508003CE01B4800EBC109D9F8140020B1012811D0EE
S31508003CF0022826D11EE0484600F0AEFB0546B5422E
S31508003D0001D2002405E0344632465146484600F0C2
S31508003D10FAFC18E0484600F09FFB0546B54201D27A
S31508003D20284600E03046044622465146484600F0FA
S31508003D30EAFC08E032465146484600F0A9FC04462B
S31508003D4001E0002400BF00BF2046BDE8F087000060
S31508003D50A41200200FB438B5044606A800906A4697
S31508003D602046059900F007F80546002000902846E9
S31508003D7038BC5DF814FB2DE9F04F99B082460D4624
S31508003D80144603A814904020159000201690CDF8EC
S31508003D9060A0179000BF2E786D1C06B9DDE0252EB1
S31508003DA079D100274FF0010900BF2E78232E12D0B3
S31508003DB02B2E0CD02D2E02D0302E10D103E047F03A
S31508003DC001076D1C0EE047F002076D1C0AE047F07C
S31508003DD004076D1C06E047F008076D1C02E04FF06B
S31508003DE0000900BF00BFB9F1000FDED14FF000088F
S31508003DF000BF2E78302E01DB392E00DD07E06D1C62
S31508003E00A6F1300008EB880100EB4108F1E700BF96
S31508003E10002013902E782E2E12D16D1C00BF2E78FE
S31508003E20302E01DB392E00DD09E06D1CA6F13000CD
S31508003E30139901EB810100EB41001390EFE700BFF6
S31508003E402E7800BF6C2E01D0682E02D16D1C2E78FC
S31508003E5000E000E0F6E700BF702E5DD008DC252EF6
S31508003E606AD0582E35D0632E09D0642E69D113E056
S31508003E70732E3CD0752E1DD0782E62D128E021688D
S31508003E80081D2060D1F8009009F0FF0B594614A8C8
S31508003E9000F0DCFB56E058E02168081D2060D1F8E8
S31508003EA00090CDE900870A22494614A8139B00F022
S31508003EB0E1FA47E02168081D2060D1F80090CDE9B5
S31508003EC000870A22494614A8139B00F049FB39E0EB
S31508003ED000BF2168081D2060D1F80090CDE9008751
S31508003EE01022494614A8139B00F03AFB2AE02168E1
S31508003EF0081D2060D1F800B000BF9BF800600BF1E8
S31508003F00010B06B906E0314614A800F09FFB179886
S31508003F100028F2DA00BF15E02168081D2060D1F8F4
S31508003F200090002008210B461022CDE900104946D2
S31508003F3014A800F015FB05E0252114A800F086FB5F
S31508003F4000E000BF00BF6D1C03E0314614A800F076
S31508003F507DFB17980028BFF61EAF00BF17980028EC
S31508003F600ADD169820B103A95046169AFFF78CFE6B
S31508003F70DDE9161008441790179819B0BDE8F08FB8
S31508003F80704700000348006840F470000149086063
S31508003F907047000088ED00E070B50546AC6B002060
S31508003FA0E085E0842046FDF79CF970BD0168C96884
S31508003FB021F490710268D1600168496921F0010114
S31508003FC002685161016B012905D10168C96821F0B0
S31508003FD010010268D160202180F83E10002101639B
S31508003FE0704710B504462068C06820F04000216874
S31508003FF0C860202084F83D002046FDF7A9FB002074
S3150800400010BD70B5044694F83E00222856D1A06823
S31508004010B0F5805F0CD1206950B90025A66A2068E2
S315080040204068C0F308003080A06A801CA06215E0D2
S31508004030A56A0026A068B0F5805F03D0A06828B9F5
S31508004040206918B920684068287004E0206840682C
S3150800405000F07F002870A06A401CA062E08D401E18
S3150800406080B2E08540BB2068C06820F02000216847
S31508004070C8602068C06820F480702168C86020681D
S31508004080406920F0010021684861202084F83E003C
S31508004090206B01280AD12068C06820F0100021682A
S315080040A0C860A18D2046FDF71BF902E02046FDF702
S315080040B00BFB0020206370BD0020FCE70220FAE716
S315080040C02DE9F84F04462068006920F44050E1685D
S315080040D00843216808612169A068084361690843A3
S315080040E0E169084300902068C06849F20C6188437A
S315080040F0009908432168C8602068406920F4407028
S31508004100A16908432168486176492068884203D036
S3150800411075492068884203D1FCF7FEFD814602E016
S31508004120FCF7EAFD8146E069B0F5004F6CD1022044
S315080041306168A0FB015003461920A9FB00700146DF
S315080041402A463846FCF7E3F86421B0FBF1F04FEA5B
S31508004150001A02206168A0FB01510B461920A9FB31
S3150800416000712A463846FCF7D2F883460220616871
S31508004170A0FB015003461920A9FB00712A463846C0
S31508004180FCF7C5F86421B0FBF1F000EBC00101EBC8
S315080041900010ABEB8000322101EBC0006421B0FBBC
S315080041A0F1F000F0F8000AEB400A02206168A0FB73
S315080041B0015003461920A9FB007001462A463846D5
S315080041C0FCF7A5F8834602206168A0FB0150034668
S315080041D01920A9FB00712A463846FCF798F864218D
S315080041E0B0FBF1F000EBC00101EB0010ABEB800077
S315080041F0322101EBC0006421B0FBF1F000F00700AA
S315080042005044216888606AE004206168A0FB015078
S3150800421003461920A9FB007001462A463846FCF7D2
S3150800422076F8824604206168A0FB015003461920EF
S31508004230A9FB007001462A463846FCF768F864214F
S31508004240B0FBF1F000EBC00101EB0010AAEB800017
S31508004250322101EB00106421B0FBF1F000F0F00A06
S3150800426004206168A0FB017003461920A9FB0051D0
S315080042703A462846FCF74BF86421B0FBF1F00AEB06
S31508004280001A04206168A0FB01510B461920A9FBFE
S3150800429000712A463846FCF73AF8834604206168D6
S315080042A0A0FB015003461920A9FB007001462A46C7
S315080042B03846FCF72CF86421B0FBF1F000EBC0019E
S315080042C001EB0010ABEB8000322101EB00106421FA
S315080042D0B0FBF1F000F00F00504421688860BDE89B
S315080042E0F88F0000001001400014014010B5034685
S315080042F099629A85DA8500201864222083F83E00A0
S3150800430000BF002083F83C0000BF1868C06840F46E
S3150800431080701C68E0601868406940F001001C68FD
S3150800432060611868C06840F020001C68E0600020E2
S3150800433010BD014691F83D00212828D18868B0F5BE
S31508004340805F0BD1086948B90A6A1088C0F308006B
S315080043500B685860086A801C086205E00B6A581CDE
S31508004360086218780B685860C88C401E80B2C884EA
S3150800437058B90868C06820F080000B68D8600868DB
S31508004380C06840F040000B68D860002070470220E3
S31508004390FCE7000070B500240F4D1048FCF7ACFF91
S315080043A000BF03E0641CAC4200D904E00B48FCF7EC
S315080043B099FF2028F6D100BF002403E0641CAC4214
S315080043C000D906E0012206490448FDF75BF90028F2
S315080043D0F4D100BF70BD0000FFFF0100EC0F002004
S315080043E05E0E002000BFFEE710B5124C02202061C9
S315080043F0606111A0A0611349E1614FF480612162F7
S315080044000021A1626162E1620BA0A0640E49E16429
S31508004410102121650021A1656165E1650BA1E01DFB
S31508004420FBF7ECFF0AA12046FBF7E8FF2020A07166
S3150800443010BD00008C1200205465726D696E616CA7
S3150800444000000000041300200417002052545400F2
S31508004450534547474552000010B501460A69CB68DF
S315080044609A4204D88C68641EE41AA01801E0D41A8B
S31508004470601E10BD2DE9FC5F06460F46924698461B
S31508004480DDE90C45002F01DA784200E0384683461C
S315080044904FF0010903E09BFBFAFB09F10109D3453B
S315080044A0F9DAC84500D9C14634B1002F03DB05F057
S315080044B00400042800D1641E05F0020010B1B8F10A
S315080044C0000F11D005F0010070B96CB108E0641E48
S315080044D02021304600F0BAF8F068002800DA02E039
S315080044E00CB1A145F3D300BFF068002836DB002FD6
S315080044F005DA7F422D21304600F0A8F807E005F0DE
S315080045000400042803D12B21304600F09FF8F068F8
S31508004510002823DB05F00200022814D105F001006B
S3150800452088B9B8F1000F0ED16CB108E0641E3021CD
S31508004530304600F08BF8F068002800DA02E00CB18B
S31508004540A145F3D300BFF068002807DB434652466F
S3150800455039463046CDE9004500F002F8BDE8FC9F33
S315080045602DE9FC5F8046894615461E460C9CCDF80B
S3150800457004900127BB4605E00198B0FBF5F00190D1
S315080045800BF1010B0198A842F6D25E4500D9B34655
S315080045900D9800F00100D0B9CCB10D9800F00200DA
S315080045A0022803D116B93020009001E0202000909F
S315080045B009E0641E4046009900F048F8D8F80C0057
S315080045C0002800DA02E00CB1A345F2D300BFD8F800
S315080045D00C00002835DB09E0012E01D9761E04E01F
S315080045E0B9FBF7FAAA4500D201E06F43F4E700BF2A
S315080045F000BFB9FBF7FA0AFB1799134810F80A1017
S31508004600404600F023F8D8F80C00002800DA03E04A
S31508004610B7FBF5F7002FECD100BF0D9800F00100AD
S3150800462078B174B109E0641E2021404600F00EF806
S31508004630D8F80C00002800DA02E00CB1A345F2D342
S3150800464000BFBDE8FC9F0000FC4B000870B504469F
S315080046500E46A568681C6168814206D320684655DF
S31508004660681CA060E068401CE060D4E9011088423C
S315080046700DD1A26821682069FFF706FBA168884268
S3150800468003D04FF0FF30E06001E00020A06070BD6D
S315080046902DE9F05F0446894617464FF0000AE5689B
S315080046A000BFD4F81080A84503D9A8EB0500461E1C
S315080046B004E0A5EB0800401CA1680E1AA068401B80
S315080046C0B04201D9304601E0A068401B0646BE420A
S315080046D001D2304600E038460646606800EB050B16
S315080046E0324649465846FBF7ADFEB244B144BF1BB5
S315080046F03544A068A84200D10025E560002FD0D136
S315080047005046BDE8F09F2DE9F04704468946154610
S31508004710E668A068871BAF420AD9606800EB060AFC
S315080047202A4649465046FBF78DFE7019E06014E0AC
S31508004730B846606800EB060A424649465046FBF70B
S3150800474081FEA5EB0708D4F804A009EB0701424649
S315080047505046FBF777FEC4F80C80BDE8F0870000EA
S3150800476002480068C0F30220704700000CED00E024
S3150800477010B5002804DB0A07130E054A135406E091
S315080047800A07140E034A00F00F031B1FD45410BD6A
S3150800479000E400E018ED00E000BF704770B58AB08D
S315080047A004460D4604B3208864281DDA208A0A21A7
S315080047B0B0FBF1F609A8032100220592CDE90621EE
S315080047C00890208AE169CDE90116CDE90302207A2D
S315080047D000902346064A29466068FDF7B1FB218802
S315080047E0044840F8214000BF38460AB070BD0000B2
S315080047F0F94A00083410002010B5044600204FF08E
S31508004800E02108610420FCF73DFD0148046010BD65
S31508004810600E002070B506460C460025304600F0AE
S315080048201DF80546A54203D2601B00F005F802E014
S31508004830012000F001F870BD38B504466A4600212B
S315080048402046FDF75BFE38BD02460020914201D3A3
S31508004850881A02E0C2F1FF335818704770B504464B
S3150800486000F008F8064631462046FFF7EDFF0546F4
S31508004870284670BD08B56846FDF79EFE08BD0000CF
S3150800488000B587B000BF00BF00200190204800682F
S3150800489040F020001E4908600846006800F0200025
S315080048A0019000BF00BF00BF00BF00BF00200190FD
S315080048B00846006840F0200008600846006800F0D6
S315080048C02000019000BF00BF00BF481502900120DC
S315080048D0039004900220059002A90E48FBF784FF76
S315080048E04FF48060029002A90A48FBF77DFF00BFDB
S315080048F0012251020748FCF783F800BF00BF0122D6
S3150800490091020448FCF77CF800BF07B000BD000020
S31508004910303802400014024038B5FBF7CDFC00BF22
S31508004920FFF7A8FF04460D4B22460DA10020FFF70E
S3150800493011FA0EA10020FFF70DFA00BF6846FCF732
S315080049400FFF0EA11248FFF729FF12A11648FFF71D
S3150800495025FF6846FDF70EFA002038BDBE4B000855
S3150800496025642025733E3E2000000000424D53205A
S315080049707374617274200D0A00000000706F6C6C0D
S315080049805F73746172745F7461736B310000000049
S31508004990080E0020706F6C6C5F73746172745F74BC
S315080049A061736B3200000000300E002010B504461B
S315080049B0204600F089F810BD10B5FCF733F8072338
S315080049C0022208214FF4A87000F010F8A820FFF77B
S315080049D013FF4FF4E13000F0D1F8FFF751FF10BD97
S315080049E010B50446204600F07BF810BD2DE9F041CD
S315080049F092B080460C4615461E460027302106A86A
S31508004A00FBF765FD142101A8FBF761FD00BF002037
S31508004A1000902A48006840F08050284908600846F7
S31508004A20006800F08050009000BF00BF00BF002063
S31508004A3000902348006840F48040214908600846F1
S31508004A40006800F48040009000BF00BF0120069077
S31508004A500004079002200C9041050D91CDF83C808A
S31508004A600E941095119606A8FCF7BEF907461FB1D5
S31508004A70012012B0BDE8F0810F20019002200290BB
S31508004A80002003904FF4A05004904FF480500590F6
S31508004A90052101A8FCF768F807460FB10120E8E7E9
S31508004AA0FBF7B4FF41F20101884205D105480068C9
S31508004AB040F48070034908600020DAE74038024075
S31508004AC000700040003C024010B5044600BF4FF499
S31508004AD000710248FBF78AFF00BF10BD00140240B0
S31508004AE010B5044600BF4FF480610248FBF77EFF0D
S31508004AF000BF10BD001402402DE9F041054600260E
S31508004B00002D26D02C46606908B16069804700BF31
S31508004B1000BFFFF7AFFE07460F4B3A460FA100202E
S31508004B20FFF718F9FFF7A6FE871B22883B460EA15A
S31508004B300020FFF70FF900BFFFF79CFE064600208E
S31508004B40E0816089A169884761893046FFF762FE7E
S31508004B50DEE7BDE8F0810000C34B00082564202588
S31508004B60733E3E20000000007461736B3A25642092
S31508004B70706572696F643A25640D0A0010B50446BB
S31508004B8009480A4908600846446000218160C160F6
S31508004B90016181610C214161FCF7D6FC01220449BF
S31508004BA00248FCF76FFD10BD00100140EC0F002015
S31508004BB05E0E00204FF04070E1EE100A70476D61FE
S31508004BC0696E007461736B5F74656D706C61746592
S31508004BD0006273705F7461736B5F626561745F779F
S31508004BE0646F670000000000000000000102030473
S31508004BF006070809000000000102030430313233B9
S31508004C00343536373839414243444546141700206F
S31508004C1006000000400000000001000014180020F3
S31508004C2080000000000200002000000000020000D2
S31508004C30141A00201E0000000A000000141C0020A0
S31508004C400A00000064000000900100004000000017
S31508004C50E80300001D0000000A000000A41D002053
S31508004C600C00000080000000000200009008000010
S31508004C70010100007856341201010000000000000E
S31508004C800000000000000000000000000000000016
S31508004C900000000000000000000000000000000006
S31508004CA000000000010101002800040000000000C7
S31508004CB000000000000000000000000000000000E6
S31508004CC000000000000000000000000001002000B5
S31508004CD0010010000C001000000000000000000099
S31508004CE000000000000000000000000000000000B6
S31508004CF000000000000000000000000000000000A6
S31508004D000000000000000000010101003000010160
S31508004D100C00200020000400040000000000000031
S31508004D200000000000000000000000000000000075
S31508004D300000000000000000000000000000000065
S31508004D400000000000000000000000000101010151
S31508004D503000010000000000000000000000000014
S31508004D600000000000000000000000000000000035
S31508004D700000000000000000000000000101010121
S31508004D8028000C0080010000040101010101010155
S31508004D9000000101C4000800010100000000000035
S31508004DA000000000000000000000000000000000F5
S31508004DB000000000000000000000000000000000E5
S31508004DC000000000000000000000000001013000A3
S31508004DD050780000C1090000F84D000800000020C6
S31508004DE0240F0000C4010008504E0008240F0020BC
S31508004DF00C1900002002000801FF01FF01FF01FF56
S31508004E0001FF01FF01FF01FF01FF01FF01FF01FF94
S31508004E1001FF01FF0116320113400613200225F493
S31508004E2001D0071A901113B9491B08AD0431822025
S31508004E30320213440D1320056BE80328411AE128B2
S31508004E408B04072801105A10641103B124F40000DA
S7050800018968
